:100000007F28B4003F202008210403197A28742097
:1000100084133408800664000D280E28A00A0319F2
:10002000A10F0B2880067A280830A6003708840024
:10003000350833193A20331D3C2036088400340932
:100040004020260803197A283318652036088400D2
:10005000A10CA00C00083404031C340680003320DB
:10006000A60B26287A283708840035088006000069
:100070008006080080043F28FF3A80054028FF3AA8
:10008000841780057A28A301A200FF30A207031C71
:10009000A307031C7A280330A100DF305120452834
:1000A000A101E83EA000A109FC30031C5A28A007CA
:1000B00003185728A0076400A10F572820186028AC
:1000C000A01C6428000064280800A201A3016C2879
:1000D000A10CA00CA20DA30DFF3E03186828230855
:1000E000A1002208A0007A28A009A109A00A0319EA
:1000F000A10A080083130313831264000800073069
:100100009F00831681133E308500FF3086008312E6
:100110003E102030BA000330BB00E6209D20640072
:1001200006083D02031998280608BD00E6209D2018
:100130000330A300E83044208F28851305130510F1
:100140000530B6008030B4000530B7004030B5004F
:100150000130B30000303E180130A000A101013091
:1001600015203A08A0003B08A1000D3015200130F1
:10017000A000A101013015200A30A000A101053026
:100180008400013001200530B6008030B400053015
:10019000B7004030B5000130B3003808A00039087E
:1001A000A1000B3015203C08A000A101073015204C
:1001B000A001A101013015200A30A000A1010530E5
:1001C0008400013001208513051305106400061A10
:1001D000EE28E330B800B9015930BC006400861A3B
:1001E000F628E330B800B9015430BC006400061BA7
:1001F000FE28E330B800B9013130BC006400861B32
:100200000629E330B800B9012C30BC0008006300B7
:020210000729BC
:02400E00701F21
:00000001FF
